:10000000B0C05BC9D3C0D2C0D1C0D0C0CFC0CEC0F9
:10001000CDC0CCC0CBC08DC9C9C0C8C0C7C0C6C0C8
:10002000C5C0C4C0C3C0C2C0C1C0C0C0BFC0BEC0C4
:10003000BDC0BCC0BBC0BAC0B9C0B8C0005EBCE2E5
:10004000613FDD83C29C7E20A3FD1F419DC3217FB4
:10005000FCA2401E5F01E3BD3E6082DC237D9FC1A8
:10006000421CFEA0E1BF5D0380DE3C62BEE0025C9C
:10007000DF81633D7C22C09E1D43A1FF4618FAA488
:1000800027799BC584DA3866E5BB5907DB85673974
:10009000BAE406581947A5FB7826C49A653BD98768
:1000A000045AB8E6A7F91B45C6987A24F8A6441A5C
:1000B00099C7257B3A6486D85B05E7B98CD2306E48
:1000C000EDB3510F4E10F2AC2F7193CD114FADF334
:1000D000702ECC92D38D6F31B2EC0E50AFF1134D28
:1000E000CE90722C6D33D18F0C52B0EE326C8ED01C
:1000F000530DEFB1F0AE4C1291CF2D73CA94762808
:10010000ABF517490856B4EA6937D58B5709EBB5F3
:1001100036688AD495CB2977F4AA4816E9B7550BE7
:1001200088D6346A2B7597C94A14F6A8742AC896DB
:10013000154BA9F7B6E80A54D7896B35010204803C
:10014000402010080402010802020201010101011D
:1001500001010102006362003936003B38003A3782
:10016000B70111241FBECFEFD2E0DEBFCDBF11E03B
:10017000A0E0B1E0E2E7FAE102C005900D92AE30F6
:10018000B107D9F721E0AEE0B1E001C01D92AB3E6E
:10019000B207E1F710E0C1EBD0E003C02197FE0108
:1001A00012DCC03BD107D1F77BDA61CC29CF80913B
:1001B00070008E7F809370002F9A81E288B962E090
:1001C00070E080E090E031D92E9A2E99FECF86B172
:1001D00027B130E0322F2227A901330F660B770BAE
:1001E0009A01AB01282B2F98809170008160809339
:1001F000700060E070E381E190E093DBCA01B90137
:100200000895CF92EF920F9385E0C82E98E0E92EE3
:1002100000E022ED41E061E089E491E014D260E485
:1002200070EC89E491E082D289E491E0BED3E0E70A
:10023000F0E084E080832F988081816080830F913B
:10024000EF90CF9008958F929F92AF92BF92CF92EE
:10025000DF92EF92FF920F931F93CF93DF9361E0B2
:1002600089E040D961E089E08BD962E370E080E009
:1002700090E0DBD888E291E07FD688E291E04DD72C
:1002800060E088E291E0D5D76B017C0160E089E015
:1002900077D960E089E026D98ADF4B015C0160E014
:1002A00071E08EE091E0A9DBCEE0D1E0FE010190AB
:1002B0000020E9F7BF01615071094AE0C401A4DBE5
:1002C00063E071E0CE018EDBFE0101900020E9F7D2
:1002D0008F010150110920E030E048EC52E4C701E1
:1002E000B601A1DAE1D9DC01CB014AE0B8018CDB2F
:1002F00089E491E05CD309900020E9F721979E0101
:100300002E50314088E1E82E01E04EE051E066E1F8
:1003100089E491E0FCD262E089E491E0BED289E414
:1003200091E043D361E088E0DDD8C0E064E670E0AE
:1003300080E090E07AD888E075D961E0892B09F0F7
:1003400060E088E01DD9CF5FC43081F768E873E1D1
:1003500080E090E0DF91CF911F910F91FF90EF909F
:10036000DF90CF90BF90AF909F908F905EC8E9E4F0
:10037000F1E083E591E09383828382E591E09583C8
:1003800084836AE08BE391E03DD46BE371E088E223
:1003900091E0F9C48627682F62956827062E669536
:1003A00066956025062E669560256770082E892F54
:1003B000669507946795902D8627069467959025F6
:1003C0008627089528B381E090E0A0E0B0E0AC017A
:1003D000BD010090DF0104C0440F551F661F771F49
:1003E0000A94D2F7422B48BB27B30090DF0104C028
:1003F000880F991FAA1FBB1F0A94D2F7822B87BBB5
:1004000061E08AE0BDD861E08AE06CD861E08BE011
:1004100069D860E08CE066D861E08DE063D880E563
:100420008093B20060E082E05DD861E082E0A8C81D
:100430008093B0008091B10087FFFCCF8091B00025
:100440000895CF92DF92EF92FF921F93CF93DF93A5
:10045000182F38B3C12CD12C7601C394B701A60153
:100460000090DF0104C0440F551F661F771F0A94D8
:10047000D2F74095242F232328BB892FD9DFC82FFB
:10048000D0E0DC2FCC27812FD3DF98B30090DF01A1
:1004900004C0CC0CDD1CEE1CFF1C0A94D2F7C92A48
:1004A000C8BA9E01282BC901DF91CF911F91FF90FF
:1004B000EF90DF90CF900895CF92DF92EF92FF926E
:1004C000CF93C82F38B3C12CD12C7601C394B70178
:1004D000A6010090DF0104C0440F551F661F771F5F
:1004E0000A94D2F74095242F232328BB892FA0DF1D
:1004F0008C2F9EDF88B30090DF0104C0CC0CDD1C84
:10050000EE1CFF1C0A94D2F7C82AC8BACF91FF90FC
:10051000EF90DF90CF900895CF9380E090E0CCDF14
:100520008091D701853081F580E090EB8ADF682FDC
:100530008091D801811104C09091DD01911172C0A8
:10054000E091D80181E08E0F8093D801F0E0E15B6B
:10055000FE4F60838091D5019091D6011BDF90936F
:10056000D6018093D501809152012091D80190E06D
:10057000059630E0821793070CF45FC08091D80194
:10058000863808F05AC05DC08091D70187FF1AC035
:10059000E09152018091D70191E0980F9093D7019B
:1005A000EC5F8E0FE82FF0E0E15BFE4FC0818091A1
:1005B000D5019091D6016C2FEDDE9093D6018093FA
:1005C000D5012CC08091D70191E0980F9093D7016D
:1005D0008330F1F054F48823A9F08130E1F4809164
:1005E000D5019091D601C92F19C08930B1F08A3058
:1005F00091F4C091DD01909152018DEF891B8093A0
:10060000D7010CC08091D5019091D601C82F06C0AA
:100610008DE092E851DFCAEA01C0CDE28C2F90E074
:1006200098540DC0E091D80181E08E0F8093D801DD
:10063000F0E0E15BFE4F908383CF8DE092E8CF91B5
:100640003BCFCF910895EF920F93CF93C42F32E019
:100650003093DF016093DE012093DD01B3DE80E0A3
:1006600090E02ADF85E092E827DF80E098EB24DF46
:1006700082E0D8D7892B19F480E090E0F8CF8C2F56
:1006800090E024E0880F991F2A95E1F7876C906825
:1006900013DF80E496EA10DF8E2D90E09A530CDF92
:1006A00082EA94E909DF8CEA92EC06DF8091DD01B1
:1006B000882341F083E89AECFFDE8091DD0190E031
:1006C0009E6C05C08BE89AECF7DE8DE29EECF4DEC2
:1006D00083E894ECF1DE083028F4802F90E0806508
:1006E000986902C087E598E9E7DE87E79CECE4DEDD
:1006F00080E090EEE1DE80E098ECDEDE83E490ECDA
:10070000DBDE84E08093D7018091DE01882349F00D
:1007100040E050E06CE872E080E0CF910F91EF9004
:10072000B1C580E0CF910F91EF90BDC59BB79F7B86
:100730009BBFCB0186DE2BB720642BBF08951092A0
:1007400052011092D8018FEF9FEF9093D6018093C2
:10075000D5016091DD01662329F01CDE9093D6015E
:100760008093D50185E08093D7018DED92E8A4CEEA
:10077000FC018091D701853039F5209152014091DB
:10078000D80130E02B5F3F4F50E02417350724F0AD
:100790008091D8018638C0F084E08093D7018091A1
:1007A0005201813830F081E090E09093D60180933F
:1007B000D501909150019F7779F0909150019F77EA
:1007C0008091DE01981741F08091D701843011F4B7
:1007D000CF01B5DF80E008958091D5019091D601D9
:1007E000892B41F40190F081E02D309719F080E0E1
:1007F00009950BC08FEF9FEFDC018093D901909397
:10080000DA01A093DB01B093DC0181E008958091CF
:10081000D701853079F48091D80181110BC008DEB1
:1008200080FD08C08DE092E847DE84E08093D70128
:1008300081E0089580E00895FC01211102C090E05C
:1008400001C090E8692B609350019091DE01411145
:1008500002C020E001C020E8922B9093510101904A
:10086000F081E02D309711F081E009958FEF9FEF37
:100870009093D6018093D5018091D5019091D601B6
:100880006091DD0187DD9093D6018093D50186E0EC
:100890008093D7018DE392E80FCE8091D701843009
:1008A000B9F06623D1F385B7877E633021F06230DB
:1008B00021F090E003C090E101C098E1892B85BF51
:1008C00085B7806285BF889585B78F7D85BFE5CF69
:1008D0000895CF92EF920F931F93CF93DF93EC0184
:1008E000162FBA0120935201422F50E083E591E088
:1008F00070D82E2D402F612FCE019EDF6C2DCE01A2
:10090000DF91CF911F910F91EF90CF90C6CF8F9233
:100910009F92AF92BF92CF92EF920F93CF93DF93BC
:1009200000D0CDB7DEB74C015A01C4012A836983D8
:100930006EDF2A816981811107C0C4012A8369831E
:1009400017DF69812A81F1CFCE2CE12CA501C401EA
:10095000C0DF0F900F90DF91CF910F91EF90CF906C
:10096000BF90AF909F908F9008951F93CF93DF9388
:10097000EC01162F67FF03C06DE072E80DC0062E74
:10098000000C770B756ED2DE65E072E8CE01CEDE2C
:10099000112321F067E072E8CE01C8DE84E0809385
:1009A000D701DF91CF911F91089560E0DECF6FEF07
:1009B000DCCFFF920F931F93CF93DF93FC01008155
:1009C000C181D281F8948981F02EF0948F2189839E
:1009D00078941DE7115009F182E090E04AD58881B2
:1009E0008023C1F3F8948A818F218A838981802BA7
:1009F0008983789480EE91E03CD5F8948981F8223F
:100A0000F98286E490E035D58881082311E009F069
:100A100010E078948AE991E02CD5812FDF91CF9175
:100A20001F910F91FF9008951F93CF93DF93FC01C7
:100A30001081C181D281812F809560FF11C0F8940F
:100A40009A8189238A838981812B89838AE090E036
:100A500010D58A81182B1A83789487E390E010C010
:100A6000F8949A8189238A838981812B898381E4FF
:100A700090E0FFD48A81182B1A83789485E090E067
:100A8000DF91CF911F91F5C40F931F93CF93DF9305
:100A9000FC011081C181D281F8948981812B8983E5
:100AA0008A81012F009580238A8383E090E0E1D43E
:100AB0008981082309838AE090E0DBD4C881789497
:100AC00085E390E0D6D41C2381E009F480E0DF9137
:100AD000CF911F910F910895CF92DF92EF92FF92E5
:100AE0000F931F93CF93DF931F92CDB7DEB76C01A7
:100AF000E62E08E010E0FF24F39461E08F2D8E21B4
:100B000009F460E0C60149838FDFFF0C0150110931
:100B100049810115110589F7411115C0F894D601D5
:100B20001196ED91FC91129791818C91809589237A
:100B300081831196ED91FC91129792818C91809511
:100B40008923828378940F90DF91CF911F910F9129
:100B5000FF90EF90DF90CF900895EF92FF920F9368
:100B60001F93CF93DF937C0108E010E0C0E0D1E059
:100B7000C7018ADF8111CD2BDD0F01501109C1F7AB
:100B80008C2FDF91CF911F910F91FF90EF900895DF
:100B9000CF92DF92EF92FF920F931F93CF93DF9349
:100BA0001F92CDB7DEB78C01F62E40E065E5798364
:100BB00093DFCF2C7981D72E760188E0E80EF11CE7
:100BC000F60161916F0140E0C80186DFCE14DF04B9
:100BD000B9F70F90DF91CF911F910F91FF90EF9098
:100BE000DF90CF90089540E06CEC76CFFC01138647
:100BF00015861486DC011B9633961E92AE17BF072E
:100C0000E1F708950F931F93CF938C01C62F60E0F7
:100C10008C2F68D46C2F70E0FB01E45CFE4FE491F4
:100C2000D801EC93FB01E85BFE4FE491F0E0E95A58
:100C3000FE4FE491F0E01296FC93EE931197C801F9
:100C4000CF911F910F91D2CFAF92BF92CF92DF92EF
:100C5000EF92FF920F931F93CF93DF931F92CDB725
:100C6000DEB75C01D62EE72EFC018585811106C01A
:100C7000C50149839EDE4981811106C0F5011386B5
:100C80001586148680E065C0442319F040E060EFCB
:100C900002C040E06CEEC5011FDF01E0F12CC12C69
:100CA00011E0C501F1DE682FC5016983EDDE6981C0
:100CB000613019F48130B9F431C04F2D50E0681320
:100CC0001BC0F5018385181730F4E40FF51F8381ED
:100CD000802349F402C0181731F060E0193058F44D
:100CE000F501148708C0F501EF0DF11D8381802BFC
:100CF000838361E009C0C12EF501E40FF51F9381E4
:100D0000802F809589238383C5018EDE1F5F000FAE
:100D100011F4F39401E0F7E0FF1518F6113408F42C
:100D2000ADCFF501C386C11002C081E08587F50112
:100D30008381882309F4A2CFD5011396ED2DFE2DD2
:100D40009501255F3F4F8D918193A217B307D9F786
:100D500081E00F90DF91CF911F910F91FF90EF9065
:100D6000DF90CF90BF90AF900895DC01E0E061503C
:100D700038F08D91E827F0E0E45CFF4FE491F7CF85
:100D80008E2F08950895FC0182EC96E0928B818B62
:100D9000768365831482108289E0818381E0828377
:100DA00083830895CF93DF93EB0167E0CE01DDDF0E
:100DB00091E02F81821390E0892FDF91CF910895E8
:100DC000EF92FF920F931F93CF93DF938C017B01E0
:100DD000D42FFC018581968109DFC0E041E0B70195
:100DE000F8018581968130DF882351F0CD1305C04D
:100DF000B701C801D7DF811104C0CF5FDC1770F7DE
:100E000080E0DF91CF911F910F91FF90EF900895B7
:100E1000CF92DF92EF92FF920F931F93CF93DF93C6
:100E200000D0CDB7DEB78C017A01FC0185819681B7
:100E300069837A83BEDD69817A818823F9F0F801BC
:100E400085819681A5DE40E06EEBF8018581968173
:100E500043DE6701F9E0EF0EF11CF8018581968110
:100E60007CDEF60181936F01EE15FF05B1F7F80105
:100E7000858196819EDD91E0813009F090E0892F97
:100E80000F900F90DF91CF911F910F91FF90EF90F6
:100E9000DF90CF900895CF93DF93EA01B9DF8823E5
:100EA00031F068E0CE0161DF91E02885821390E0A7
:100EB000892FDF91CF910895EF92FF921F93CF93E7
:100EC000DF9300D0CDB7DEB77C01FC018581968130
:100ED00069837A836EDD69817A81F70185819681E4
:100EE00057DE40E064EBF70185819681F5DDF7017F
:100EF00085819681C9DD182FF7018581968159DD9D
:100F000081E0111180E00F900F90DF91CF911F9140
:100F1000FF90EF900895CF93DF93CDB7DEB7299779
:100F20000FB6F894DEBF0FBECDBFFB01208120318C
:100F3000C9F0AE014F5F5F4FAEDF882389F08D812E
:100F40008F3361F020F48F3159F489E00CC08F3574
:100F500019F08F3739F004C08BE005C08AE003C078
:100F600080E001C08CE029960FB6F894DEBF0FBE7A
:100F7000CDBFDF91CF910895FF920F931F93CF9331
:100F8000DF93CDB7DEB728970FB6F894DEBF0FBE5C
:100F9000CDBF8C01FC018581968128DEF801148289
:100FA00041E0BE016F5F7F4FF801858196814CDE85
:100FB000882369F1BE016F5F7F4FC801F3DE88238C
:100FC00079F3F8018081811107C0BE016F5F7F4F07
:100FD000C80172DF811117C0F801F180BE016F5F97
:100FE0007F4FC80198DF8F1518F4F801818105C083
:100FF000BE016F5F7F4FC8018EDFF801818384815E
:101000008F5F8483CDCF81E0F8018083E5CF289680
:101010000FB6F894DEBF0FBECDBFDF91CF911F9109
:101020000F91FF900895CF93DF93CDB7DEB7299747
:101030000FB6F894DEBF0FBECDBFAE014F5F5F4F5E
:10104000E7DE81E09981911101C080E029960FB619
:10105000F894DEBF0FBECDBFDF91CF9108958F9280
:101060009F92AF92BF92CF92DF92EF92FF920F9337
:101070001F93CF93DF93EC01E7EFE60FE33040F4EB
:10108000F0E0EE0FFF1FE95FFE4FC080D18004C08B
:101090008EEEC82E82E0D82E4115510501F18B81CC
:1010A0008823E9F0888181111AC08A018CD14B0113
:1010B0005C010D2C000CEE08FF08B801CE01B3DF77
:1010C00081111EC080D1DC01CB018C199D09AE09B4
:1010D000BF0988159905AA05BB0578F311C0B601AB
:1010E000DD0C880B990BDF91CF911F910F91FF9031
:1010F000EF90DF90CF90BF90AF909F908F9095C171
:10110000DF91CF911F910F91FF90EF90DF90CF90E3
:10111000BF90AF909F908F900895CF93DF93EC0195
:101120008D819E8146DC8D819E815DDD488164E4F8
:101130008D819E81D1DC8A81882339F040E050E0A6
:101140006981CE01DF91CF918ACFDF91CF91089550
:10115000FA01208130E0A3E0220F331FAA95E1F7C6
:10116000818190E0982F8827990F990F990F282B4C
:10117000392BDB018C918031B9F4678170E0868175
:10118000AB01481B5109CA019695982F882797955E
:101190008795B4D360517109207F53E0220F331F2C
:1011A0005A95E1F7260F371FC9010895EF92FF9274
:1011B0000F931F93CF93DF93CDB7DEB729970FB669
:1011C000F894DEBF0FBECDBF8C017B01AE014F5F37
:1011D0005F4F61DE882339F0AE014F5F5F4FB7018B
:1011E000C801B6DF02C080E894EE29960FB6F894E5
:1011F000DEBF0FBECDBFDF91CF911F910F91FF904A
:10120000EF900895813824EE920764F0BC01072E18
:10121000000C880B990B7BD220E030E040E05CE3CF
:1012200002D3089560E070E08EEF92EC0895BEDF87
:10123000E9CF0F931F93CF93DF93CDB7DEB72897F6
:101240000FB6F894DEBF0FBECDBF8C01462FBE0196
:101250006F5F7F4FB5DD882331F0BE016F5F7F4F39
:10126000C801E5DF04C060E070E08EEF92EC2896E4
:101270000FB6F894DEBF0FBECDBFDF91CF911F91A7
:101280000F91089581110EC08FB7F8947093E1010A
:101290006093E0018FBF85B78C7F482B45BF8BB72C
:1012A00080648BBF0895811107C08BB78F7B8BBF84
:1012B0001092E1011092E00108951F920F920FB673
:1012C0000F9211242F933F934F935F936F937F93CC
:1012D0008F939F93AF93BF93EF93FF938091E00120
:1012E0009091E101892B29F0E091E001F091E10179
:1012F0000995FF91EF91BF91AF919F918F917F9150
:101300006F915F914F913F912F910F900FBE0F9072
:101310001F9018958EB5887F8EBD8FB58C7F8160AC
:101320008FBD8EB5877E8EBD8EB5887F83608EBD66
:1013300008951F920F920FB60F9211242F933F938F
:101340008F939F93AF93BF938091E3019091E401BA
:10135000A091E501B091E6013091E20126E0230F72
:101360002D3730F029E8230F0396A11DB11D03C0CE
:101370000296A11DB11D2093E2018093E301909399
:10138000E401A093E501B093E6018091E70190911B
:10139000E801A091E901B091EA010196A11DB11DFA
:1013A0008093E7019093E801A093E901B093EA01EB
:1013B000BF91AF919F918F913F912F910F900FBE51
:1013C0000F901F9018952FB7F8946091E3017091DA
:1013D000E4018091E5019091E6012FBF08953FB7A8
:1013E000F8948091E7019091E801A091E901B09112
:1013F000EA0122B708B600FE05C02F3F19F001969A
:10140000A11DB11D3FBFBA2FA92F982F8827820F8A
:10141000911DA11DB11DBC01CD0143E0660F771FD9
:10142000881F991F4A95D1F70895CF92DF92EF92C6
:10143000FF92CF93DF936B017C01D1DFEB01C114ED
:10144000D104E104F10471F0CADF6C1B7D0B683E2E
:101450007340A8F381E0C81AD108E108F108C85127
:10146000DC4FEDCFDF91CF91FF90EF90DF90CF90E9
:1014700008958330910528F0880F991F04970197EC
:10148000F1F70895789480B7836080BF83B7877F32
:1014900083BF83B7887F836083BF89B7816089BF3B
:1014A00039DFE9ECF0E08081887F808380E1809300
:1014B000670084EA809368008CEF80936600AAEC52
:1014C000B0E08C918C7F81608C938081877E80835B
:1014D0008081887F8360808385B1887F866085B9BD
:1014E0002F9A0895CF93DF93A82FB0E0FD01E45C1D
:1014F000FE4F9491FD01E85BFE4FA491AA2309F4ED
:101500003CC0B0E0FD01E35AFE4FE491CE2FD0E0A5
:10151000FD01E65AFE4FE4912E2F30E0FD01EC5A1A
:10152000FE4FA491B0E0892F809561110DC04FB797
:10153000F894988198239883F90190819823908357
:101540009C9189238C930EC0623071F44FB7F8944C
:10155000588185238883F9018081892B8083EC91D0
:101560009E2B9C934FBF09C02FB7F8943C918323C7
:101570008C93E8819E2B98832FBFDF91CF910895A4
:10158000CF93DF93A82FB0E0FD01E45CFE4F949170
:10159000FD01E85BFE4FA491AA2309F440C0863008
:1015A00019F480B78F7304C0853021F480B78F7C25
:1015B00080BF18C0843019F48FB58F7304C0873092
:1015C00021F48FB58F7C8FBD0DC0823021F48091C6
:1015D000CA008F7305C0833029F48091CA008F7CC4
:1015E0008093CA00B0E0FD01E65AFE4FC491D0E0FE
:1015F000FD01EC5AFE4FA491B0E0892F80952FB7E2
:10160000611105C0F89498819823988304C0F894D8
:10161000E881E92BE8839C9189238C932FBFDF918C
:10162000CF910895282F30E0F901E45CFE4F9491AA
:10163000F901E85BFE4FE491EE2379F1863019F46D
:1016400080B78F7304C0853021F480B78F7C80BF52
:1016500018C0843019F48FB58F7304C0873021F41B
:101660008FB58F7C8FBD0DC0823021F48091CA0070
:101670008F7305C0833029F48091CA008F7C8093DA
:10168000CA00F0E0E95AFE4FA491B0E0EC91E923E2
:1016900081E090E021F480E0089580E090E00895FA
:1016A000F1DEAFD5D0D5FECF04D06894B111B5C06E
:1016B000089598D088F09F5790F0B92F9927B75187
:1016C000A0F0D1F0660F771F881F991F1AF0BA9506
:1016D000C9F712C0B13081F09FD0B1E008959CC02D
:1016E000672F782F8827B85F39F0B93FCCF38695FC
:1016F00077956795B395D9F73EF490958095709559
:1017000061957F4F8F4F9F4F0895E89409C097FBD5
:101710003EF490958095709561957F4F8F4F9F4FC8
:101720009923A9F0F92F96E9BB279395F69587950C
:1017300077956795B795F111F8CFFAF4BB0F11F4CF
:1017400060FF1BC06F5F7F4F8F4F9F4F16C0882376
:1017500011F096E911C0772321F09EE8872F762FAC
:1017600005C0662371F096E8862F70E060E02AF0ED
:101770009A95660F771F881FDAF7880F96958795D9
:1017800097F9089597F99F6780E870E060E0089501
:101790009FEF80EC089500240A9416161706180689
:1017A0000906089500240A94121613061406050665
:1017B0000895092E0394000C11F4882352F0BB0FF6
:1017C00040F4BF2B11F460FF04C06F5F7F4F8F4F59
:1017D0009F4F089557FD9058440F551F59F05F3F94
:1017E00071F04795880F97FB991F61F09F3F79F043
:1017F00087950895121613061406551FF2CF4695C5
:10180000F1DF08C0161617061806991FF1CF869546
:101810007105610508940895E894BB27662777272A
:10182000CB0197F908950AD0C4CFB5DF28F0BADF0D
:1018300018F0952309F0A6CFABCFEFCFCBDFA8F3FD
:101840009923D9F35523C9F3950F50E0551FAA27C3
:10185000EE27FF27BB2700240894679520F4E20FAA
:10186000F31FB41F0A1E220F331F441FAA1F6695C1
:10187000A9F7779530F4F30FB41F0A1E121E08F46F
:101880006395330F441FAA1F221F769599F78795FA
:1018900020F4B40F0A1E121E631F440FAA1F221F3A
:1018A000331F8695A9F7862F712D602D11249F5720
:1018B00050408AF0E1F088234AF0EE0FFF1FBB1F73
:1018C000661F771F881F91505040A9F79E3F510512
:1018D00070F058CFA2CF5F3FECF3983EDCF38695D3
:1018E00077956795B795F795E7959F5FC1F7FE2BBD
:1018F000880F911D9695879597F9089597FB072E68
:1019000016F4009406D077FD08D027D007FC05D048
:101910003EF4909581959F4F0895709561957F4F06
:101920000895052E97FB16F400940FD057FD05D0AF
:1019300028D007FC02D046F408C050954095309559
:1019400021953F4F4F4F5F4F08959095809570952B
:1019500061957F4F8F4F9F4F0895AA1BBB1B51E18D
:1019600007C0AA1FBB1FA617B70710F0A61BB70B0F
:10197000881F991F5A95A9F780959095BC01CD01B4
:101980000895A1E21A2EAA1BBB1BFD010DC0AA1FC0
:10199000BB1FEE1FFF1FA217B307E407F50720F0D8
:1019A000A21BB30BE40BF50B661F771F881F991F53
:1019B0001A9469F760957095809590959B01AC019C
:1019C000BD01CF010895EE0FFF1F0590F491E02DAA
:1019D0000994FB01DC0102C001900D92415050407E
:1019E000D8F70895FB01DC010D900020E9F711976D
:1019F00001900D920020E1F70895FB01DC010190B8
:101A00000D920020E1F70895BB274A3031F4992365
:101A100022F4BDE2909581959F4F01C0BB27FB0149
:101A20005527AA27880F991FAA1FA41710F0A41BD7
:101A300083955051B9F7A05DAA3308F0A95DA19331
:101A4000009779F7B111B1931192CB0100C0DC017D
:101A5000FC01672F71917723E1F7329704C07C91E5
:101A60006D9370836291AE17BF07C8F30895F89421
:021A7000FFCFA6
:0E1A7200763D0026743D005E00BC007701004A
:00000001FF
